:1000000000308A0098280000FF00030E8301A10041
:100010007F08A0000A08A8008A01A00E0408A20018
:100020007708A3007808A4007908A5007A08A6003C
:100030007B08A700831383128C308400801C222845
:100040008C183528220884002308F7002408F800BB
:100050002508F9002608FA002708FB0028088A006E
:10006000210E8300FF0E7F0E09008A1143280A101B
:100070008A100A118207013405340434063402342C
:100080000A34083409342A082907A900290807393D
:10009000B20032083720F800B2003218512806109A
:1000A00052280614831606108312B2185928861097
:1000B0005A28861483168610831232196128061175
:1000C00062280615831606118312B2196928861153
:1000D0006A2886158316861183128C108A112228AD
:1000E000B01B78283008013C031878280130B00094
:1000F0003008803A7E3C031C7F28FF30B000300877
:10010000AA00003431308400000803199628013019
:10011000F800F701F70B8A28F80B89284A30F70016
:10012000F70B902800000000800B87288A113029E7
:1001300084011F30830583161F129F121B0880390C
:100140009B0007309C001C0883120D13603083163F
:100150008F000610831206108316861083128610F5
:1001600083160611831206118316861183128611D7
:10017000831681131F129F121B08803901389B00C0
:100180001F1383121F179F1783169F1383121F14A9
:100190000030F8001F08C73978049F0094128316B6
:1001A0000611861406120030831294008316940000
:1001B0000108C7390838810083129001073083167F
:1001C0009C0005080330F700F70BE4281C08831295
:1001D0000D1383169D018312A9010030F800063823
:1001E0009200FF3083169200C03083128B04831676
:1001F0008C1483121F1DFE288316F9281E08AC01DB
:10020000AB001F15AB08031D0829AC0803190C2906
:100210002B08831692008312831686168312861E7D
:100220001E29831606168312061E1A290130B000F5
:1002300070201D29FF30B00070203E292908E63CBF
:1002400003183629831606168312061A33292F1C23
:100250003329B00170200230B000FA30B10082289A
:10026000B00B2D292F10FF30B000702029081D3C45
:10027000031C3E290130B00070202F148316F9288A
:02028000630019
:04400E003B3FFF3FF6
:00000001FF
